:03000000020444B3
:030003000202F303
:03000B00020145AA
:1000130002032D758921759852758780758DFED2DF
:100023008E223099FDC299F5993010042524F524C8
:10003300227F057E00209807DEFBDFF774FF22C2D4
:1000430098E599223098FDC298E59912002522126D
:10005300005C9006B112066E22740D120025740A1C
:100063001200252274131200252274111200252276
:10007300742012002522C3FE94415005EEC3943030
:1000830022C3EE943722EDC42C22120047120079CA
:10009300FD120047120079FC12008922540FFAC3A3
:1000A300940A5004EA243022EA243722F5F012009D
:1000B3009FFCE5F0C412009FFD221200AFED120079
:1000C30025EC1200252208E6C454F0F918E6C4FA18
:1000D300540F2908F6EA54F018F622C3E53D253DEE
:1000E300F53DE53E353EF53E227536007537007524
:1000F300380079007F101200DE5011900115C3788B
:10010300367E03E99336D4F6A308DEF7090909DF3F
:10011300E52268270384630192810096400048200A
:10012300002410001205005602002801006400009C
:100133003200001600000800000400000200000165
:100143000000C0D0C0E0C0F0C082C08375D0087585
:100153008C8B852F8A1202220525E525B40A2712E6
:1001630003C712005C052CE52CB40507752C00D2DF
:100173001AC2B712028C30180312024B752500E520
:10018300262401D4F526E526B460103019031202A3
:100193004B752600E5272401D4F527E527B4600A2B
:1001A300752700E5282401D4F528E528B4240A7529
:1001B3002800E5292401D4F5291202B1E529B5F077
:1001C3000A752901E52A2401D4F52AE52AB4130A7C
:1001D300752A01E52B2401D4F52BD083D082D0F0EE
:1001E300D0E0D0D0D28C321200731200737E019013
:1001F300070212066E78217F08E6F4F590F4F5F015
:10020300E5F033F5F0400A742D12002512007380D7
:1002130008744F120025120073DFE508DED922307F
:100223001A0FE52D04F52DB40107752D00D2B7C2C1
:100233001A227F00C2A27E50DEFED2A27E50DEFED4
:10024300DFF222540F24302212005CE5291200BD94
:10025300742D120025E52A1200BD742D1200257499
:10026300251200BDE52B1200BD120073E528120014
:10027300BD743A120025E5271200BD743A12002519
:10028300E5261200BD1201EA227833E6B40F0122FB
:1002930020B503B5291208E6B5280E08E6B5270AE6
:1002A30008E6F521F4F590220808080880DDE52A20
:1002B300C394104007E52AC394068002E52A1490EC
:1002C30002CB93F5F005F022312831303130313152
:1002D300303130317F067830E6120246F608DFF817
:1002E300227F067835E612002518DFF912005C221A
:1002F300C0D0C0E0C0F0C082C08375D01012030E1E
:10030300D083D082D0F0D0E0D0D032742A1200252E
:10031300752400D210120369120359C210E524F4A4
:10032300041200BD740012002522C0D0C0E0C0F04A
:10033300C082C08375D018C37834E63401D4F6087C
:10034300E63400D4F608E63400D4F6D083D082D065
:10035300F0D0E0D0D032E5361200BDE5351200BD55
:10036300E5341200BD22E537A2E09290A2E192911A
:10037300A2E2929212043330B7FD20B7FD1204219A
:100383004390F0E59054F0C4F53020B5FD4390F070
:10039300E59054F0C4F53120B4FD4390F0E590545A
:1003A300F0C4F5321203DEE530120025E532120007
:1003B30025E5311200250537E537B523A975370043
:1003C3007590F022C2A81203DEE530120025E53253
:1003D300120025E531120025D2A822E530B40A0522
:1003E30075302D800CB40B0575304580042430F531
:1003F30030E532B40A0575322D800CB40B05753225
:100403004580042430F532E531B40A0575312D8079
:100413000CB40B0575314580042430F531227B0182
:100423007C95DCFEDBFA227B027C95DCFEDBFA2288
:100433007BC87C95DCFEDBFA22C3E6970809E697C6
:1004430022758160752D007590FFC218C21A75253B
:1004530000752C00752F92E52EB425028027752E8A
:100463002575330F752600752730752812752929D0
:10047300752A04752B3775210075340075350075A1
:100483003600752308D2AFD2A9758901120016D29E
:10049300B9758C8B758A92D28AD2AA753700D2A885
:1004A300D28880FE3098FBC298E599B4410E1200C1
:1004B30047B45408120047B40DFA80E64420B46FE1
:1004C30002804EB474028050B47A02804FB4650245
:1004D300807DB46403020570B43F0302058EB473D8
:1004E3000302059AB4700302059FB4720302060265
:1004F300B46303020659B42F03020668B46D030202
:10050300053A1200520204A5758A92758C8BD28C1F
:1005130022C218120052808AD218808612005CE52B
:100523002F1200BD12005C743F12002512008DF5DE
:100533002F1200520204A512005CE5231200BD1223
:10054300005C743F12008DF5231200520204A59043
:10055300071112066E12008DF52812008DF5271271
:10056300008DF52612024B1200520204A5900729B2
:1005730012066E12008DF52912008DF52A12008DD8
:10058300F52B12024B1200520204A59006B4120678
:100593006E1200520204A5B2190204A5C28C900681
:1005A300E712066E12005C7833120047B43AFA126F
:1005B300008DB40002803212004712008DF6120043
:1005C300470812008DF60812008DF6087F08120006
:1005D30047120047B43003C38001D3E633F6DFEE9E
:1005E300120047B40AFA0880C0760F120047B40A13
:1005F300F89006D612066E120052D28C0204A5128F
:10060300005C7833E6B40F0890074112066E804011
:100613001200BD12007308E61200BD743A120025E1
:1006230008E61200BD12007390070212066E08E678
:100633007F0833F5F04007742D1200258005744FB1
:10064300120025120073E5F0DFE812005C0880B4A5
:100653001200520204A57521007590FF12024B127D
:1006630000520204A512030E0204A5E493B4100180
:1006730022C082C083120025D083D082A380EC0DD8
:100683000A414E414C4F472053454E4445520D0AB3
:1006930044657369676E656420627920576963688E
:1006A3006974205369726963686F74650D0A262043
:1006B300100D0A2F20747269676765722072656175
:1006C300640D0A6D206D6178206368616E6E656CE0
:1006D3000D0A1050726F6772616D2073746F7265CB
:1006E300640D0A100D0A526561647920746F2072DB
:1006F3006563656976652070726F6772616D104F0F
:100703005554505554205B312E2E385D20100D0A60
:10071300456E7465722063757272656E74207469B8
:100723006D65203E20100D0A456E74657220637559
:100733007272656E742064617465203E2010454FAB
:0A0743004610574841543F0D0A10BC
:00000001FF
